:100000000C94CD000C94F5000C94F5000C94F500C4
:100010000C94F5000C94F5000C94F5000C94F5008C
:100020000C94F5000C94F5000C94F5000C94FB0C6A
:100030000C942F110C94F5000C94F5000C94F50021
:100040000C9456140C94F5000C9462160C94F50064
:100050000C94F5000C94F5000C94F5000C94F5004C
:100060000C94F5000C94F500746F6F206D616E793F
:10007000206F70656E2066696C6573006261642034
:10008000696E707574005941414B00594545454BA7
:100090000053616D706C65207261746520746F6FC0
:1000A0002068696768210000436F6D707265737323
:1000B000696F6E206E6F7420737570706F727465E7
:1000C00064006661696C656420746F2067657420E4
:1000D0006E657720636C7573746572002021212131
:1000E0002000203F3F3F200046696C657320666F0B
:1000F000756E643A0046696C657320666F756E6450
:100100003A00436F756C646E2774206F70656E20C3
:1001100064697200436F756C646E2774206F70653C
:100120006E2066696C65737973004E6F2070617222
:10013000746974696F6E21004361726420696E692D
:10014000742E206661696C65642100000024272AF2
:10015000000025282B00002326290404040404049D
:100160000404020202020202030303030303010266
:100170000408102040800102040810200102040835
:100180001020000000070002010000030406000028
:100190000000000000007911AE1211241FBECFEF45
:1001A000D4E0DEBFCDBF11E0A0E0B1E0E0EAFEE2C6
:1001B00002C005900D92AA34B107D9F714E0AAE461
:1001C000B1E001C01D92AB38B107E1F711E0CAE917
:1001D000D1E004C02297FE010E944A17C639D10718
:1001E000C9F70E94A7120C944E170C9400000895B2
:1001F0000895CB010E941B030895FC018481958121
:100200000E94AD040895EF92FF920F931F93CF9336
:10021000DF93EB018A0179010BC0B801C7010E948D
:100220009F16009729F4CE010E94AD0481E006C01C
:10023000B701CE010E94B604882379F7DF91CF91F0
:100240001F910F91FF90EF900895EF92FF920F93FF
:100250001F93DF93CF93CDB7DEB768970FB6F894AF
:10026000DEBF0FBECDBF8C017E010894E11CF11CE6
:1002700097010E940301882319F420E030E005C0B3
:10028000B701C8010E948F089C01C90168960FB68A
:10029000F894DEBF0FBECDBFCF91DF911F910F91BC
:1002A000FF90EF900895FC01AB016481758182811C
:1002B00093810E9425010895EF92FF920F931F935F
:1002C000DF93CF93CDB7DEB768970FB6F894DEBF54
:1002D0000FBECDBF8B017E010894E11CF11CB7015C
:1002E000FC01848195810E94B604882349F04CE08A
:1002F00050E0B701C8010E94B616F801148681E0EB
:1003000068960FB6F894DEBF0FBECDBFCF91DF91D8
:100310001F910F91FF90EF900895FC0184819581CA
:100320000E94A7040895EF92FF920F931F93DF930B
:10033000CF93CDB7DEB768970FB6F894DEBF0FBE88
:10034000CDBF8C017E010894E11CF11CB701FC01BA
:10035000828193810E945905B701F80182819381BE
:100360000E944007F8019583848320E0892B09F0DF
:1003700021E0822F68960FB6F894DEBF0FBECDBF86
:10038000CF91DF911F910F91FF90EF9008950F9300
:100390001F938C01FC01808191810E946A05F80104
:1003A0009383828320E0892B09F021E0822F1F9123
:1003B0000F9108950F93CF93DF93EC0100E020E0BD
:1003C00030E040E050E06CE17BE082E69AE00E94A1
:1003D000D60899838883892B69F40FEF20E030E0F9
:1003E00040E050E06CE17BE082E69AE00E94D608B3
:1003F0009983888320E088819981892B09F021E005
:10040000822FDF91CF910F9108950E940C0A0895D9
:10041000FC01009711F0118210820895DC018C918B
:10042000853E39F1882329F1F901208131818281CA
:1004300093812817390799F444835583668377831A
:100440001B968C911B978F3011F080E205C08C9128
:100450008295880F807E805E808780E008951B965D
:100460008C918F3031F02F5F3F4F3183208381E0BB
:10047000089581E008950F931F93CF93DF938C012C
:10048000FC018081853E09F48CC0882309F489C071
:10049000E9018C899D89AE89BF890097A105B105C5
:1004A00021F44C8B5D8B6E8B7F8B209709F479C088
:1004B0000115110509F475C0F8018081882309F43C
:1004C00070C083858F3011F481E06CC0A801D80121
:1004D00080E090E0282F3C91303251F0FE01E80F8F
:1004E000F91F30832F5F019611968830910591F79F
:1004F0008881853011F485EE8883F801808580320B
:10050000B1F0FE01E20FF11D8EE28083822F8F5F3A
:100510002C5FFA019085903249F0FE01E80FF11D41
:1005200090838F5F4F5F5F4F821799F7282FFE01EF
:10053000E20FF11D1082F80183858D87938D80E095
:10054000228D30E0822B932B9F878E87258D30E084
:1005500040E050E0542F432F322F2227868D90E029
:10056000A0E0B0E0DC0199278827282B392B4A2B03
:100570005B2B848D90E0A0E0B0E0282B392B4A2B38
:100580005B2B878D90E0A0E0B0E0B82FAA279927D9
:100590008827282B392B4A2B5B2B288B398B4A8BAE
:1005A0005B8B80E0DF91CF911F910F910895DF93D6
:1005B000CF9300D0CDB7DEB7DC010097A1F1623058
:1005C000710588F1ED91FC911197660F771F80E01E
:1005D00090E016962D913D914D915C911997620F87
:1005E000731F841F951F0190F081E02D22E030E001
:1005F000AE014F5F5F4F09958823A9F09A8180E093
:10060000298130E0282B392B2115310571F08FEF2E
:10061000273F380741F0C9014096079720F08FEF38
:10062000283F380710F020E030E0C9010F900F900C
:10063000CF91DF910895FC01009711F01182108293
:1006400008952F923F924F925F926F927F928F9276
:100650009F92AF92BF92CF92DF92EF92FF920F9351
:100660001F93DF93CF93CDB7DEB72C970FB6F894D7
:10067000DEBF0FBECDBF3C0178876F835A874987A5
:10068000009709F402C1672B09F4FFC0452B09F458
:10069000FCC0DC015A96AD90BD90CD90DC905D978A
:1006A00052962D913D914D915C915597E985FA8532
:1006B000CF01A0E0B0E08A0D9B1DAC1DBD1D281729
:1006C00039074A075B0740F4B9016A197B097A8741
:1006D0006987672B09F4DCC0D301ED91FC91119778
:1006E000208931893A8329835E966D917C915F9749
:1006F0007C876B87C901A0E0B0E08B839C83AD83CE
:10070000BE83672BE1F5F3010088F189E02DFC87BA
:10071000EB87EF2B39F4A114B104C104D10409F41F
:10072000B7C0B3C0A114B104C104D10441F1860122
:1007300075012B803C804D805E80509440943094B5
:100740002094211C311C411C511C10C06B857C85E0
:10075000D3018D919C910E94D7029C878B87892B16
:1007600009F493C0E20CF31C041D151D6B817C8100
:100770008D819E81E616F7060807190738F7C6012E
:10078000B5012B813C814D815E810E940B172B01AD
:1007900089849A84D301ED91FC91A980BA80A41830
:1007A000B5088A149B0408F45401C080D1807201FA
:1007B00000E010E086899789A08DB18DE80EF91EC2
:1007C0000A1F1B1FEB85FC853297BF0180E090E07C
:1007D0003296FC87EB872B813C814D815E810E94A4
:1007E000C516E60EF71E081F191FD601ED91FC91E4
:1007F00095014F815885C801B7010995882361F19A
:100800008A189B08C501A0E0B0E0F301228D338D6A
:10081000448D558D280F391F4A1F5B1FD3015A96EF
:100820002D933D934D935C935D97C501840D951D6C
:10083000E981FA818E179F07B0F06B857C858D91D9
:100840009C910E94D7029C878B87892B51F4D301FE
:100850005F961C921E925E9749855A8548195909E0
:1008600019C0442455242B853C85F301378F268FEE
:100870008114910439F06F8178856A0D7B1D78872A
:100880006F8388CF49855A8505C04FEF5FEF02C05F
:1008900040E050E0CA012C960FB6F894DEBF0FBEC0
:1008A000CDBFCF91DF911F910F91FF90EF90DF901F
:1008B000CF90BF90AF909F908F907F906F905F9000
:1008C0004F903F902F900895CF93DF93FC01EB0161
:1008D0000097C9F161157105B1F1828D938DA48DD9
:1008E000B58D413051F0413018F0423061F50AC009
:1008F000288139814A815B8111C0288139814A81EF
:100900005B8108C0288139814A815B818289938912
:10091000A489B589280F391F4A1F5B1F82899389D3
:10092000A489B58982179307A407B50760F0228FC1
:10093000338F448F558F178E168E288339834A83C1
:100940005B8381E001C080E0DF91CF910895FC01DD
:10095000009711F0118210820895FC01009711F4A4
:1009600080E00895138E128E81E008952F923F92B9
:100970004F925F926F927F928F929F92AF92BF92AF
:10098000CF92DF92EF92FF920F931F93DF93CF935B
:10099000CDB7DEB7A9970FB6F894DEBF0FBECDBFB7
:1009A0003C012B01009709F44AC06115710509F457
:1009B00046C0FC0180899189892B09F040C0228DB5
:1009C000338DA081B1811097B9F1ED91FC91119710
:1009D00022803380AE014F5F5F4F89E0FA011192B0
:1009E0008A95E9F73C832B8352966D917D918D9189
:1009F0009C91559756960D911C915797061B170B76
:100A00006A012EE0E22E22E0F22E20E230E0AE017A
:100A1000465F5F4FF1010995882371F08D809E80BC
:100A2000AF80B88481149104A104B10429F021C0DD
:100A3000F20180818823A9F5F301138E128E80E0E4
:100A4000A9960FB6F894DEBF0FBECDBFCF91DF9150
:100A50001F910F91FF90EF90DF90CF90BF90AF90DC
:100A60009F908F907F906F905F904F903F902F90CE
:100A7000089588E1F20111928A95E9F709856201EA
:100A80009BE3E92E92E0F92E10E020E230E0AE0187
:100A9000465F5F4FC501B401F1010995882361F2FA
:100AA000C7CFF301828D938D0196938F828F81E062
:100AB000C7CFFB01892B61F06115710549F088E111
:100AC000DB011D928A95E9F780E1858781E0089531
:100AD00080E008952F923F924F925F926F927F92A3
:100AE0008F929F92AF92BF92CF92DF92EF92FF923E
:100AF0000F931F93DF93CF93CDB7DEB7E0970FB679
:100B0000F894DEBF0FBECDBF6C01009709F490C111
:100B1000ABC1E2EAF1E08AE1DF011D928A95E9F7D3
:100B2000D092A301C092A201D60119962D913D91B8
:100B30004D915C911C9719E0220F331F441F551FE4
:100B40001A95D1F72AA33BA34CA35DA3CA01B9010F
:100B5000655F7F4F8F4F9F4FED91FC9129E130E012
:100B6000AE014F5F5F4F0995882309F484C1A980C6
:100B70004A80BB81BEA30C81FD801E813F815884C9
:100B800069847A849D8580E02C85E22FF0E0E82B53
:100B9000F92B8E883F88288DE98C309709F46BC13A
:100BA000432D50E060E070E0962F852F742F66276C
:100BB00069A77AA78BA79CA7822F90E0A0E0B0E05E
:100BC000BC015527442789A59AA5ABA5BCA5842BB4
:100BD000952BA62BB72B482D50E060E070E0842BBE
:100BE000952BA62BB72B89A79AA7ABA7BCA78E2DB1
:100BF00090E0A0E0B0E0782F66275527442789A52C
:100C00009AA5ABA5BCA5842B952BA62BB72B89A7A2
:100C10009AA7ABA7BCA70097A105B10589F4972DAA
:100C200080E0662D70E0682B792B6115710509F461
:100C300022C1CB01A0E0B0E089A79AA7ABA7BCA7CF
:100C4000942D80E02A2C3324282A392A952D80E0FF
:100C5000A32FB0E0A82BB92BB8A7AFA39F2D80E09E
:100C6000202F30E0822B932B9C0140E050E02A8F14
:100C70003B8F4C8F5D8FBF0180E090E0212F30E0F3
:100C800040E050E00E94C5166E8F7F8F88A399A325
:100C9000E9A4FAA40BA51CA54A8D5B8D6C8D7D8DF6
:100CA000E41AF50A060B170B6E8D7F8D88A199A1AA
:100CB000E61AF70A080B190BC10101972FA138A5F5
:100CC000B5E0220F331FBA95E1F7820F931FB101F0
:100CD0000E94E41680E090E0E61AF70A080B190B70
:100CE0007EA1272F30E040E050E0C801B7010E940C
:100CF0000B1729013A01D301C201855F9F40A04033
:100D0000B0408050904FA040B04008F0B4C086E0A2
:100D1000D60118968C93A4EA8A2EA1E09A2E88E137
:100D2000F40111928A95E9F75101CC24DD2469A5DB
:100D30007AA58BA59CA5A60195010E94C516609376
:100D4000A4017093A5018093A6019093A701C60109
:100D5000B5012A8D3B8D4C8D5D8D0E94C5167B01A2
:100D60008C012AA13BA14CA15DA1E20EF31E041F40
:100D7000151FE092A801F092A9010093AA01109317
:100D8000AB0142E050E060E070E0440E551E661E8C
:100D9000771E440C551C661C771C4092AC01509287
:100DA000AD016092AE017092AF013092B10120921C
:100DB000B0015EA1852F90E0BC01269EC001279E58
:100DC000900D369E900D11249093B3018093B20143
:100DD0006E8D7F8D88A199A1A60195010E94C516EF
:100DE0006E0D7F1D801F911F6093B4017093B5013C
:100DF0008093B6019093B701AFA1B8A59D0140E0E3
:100E000050E0E5E0220F331F441F551FEA95D1F74C
:100E1000620F731F841F951F6093B8017093B9010F
:100E20008093BA019093BB0194012250304002C0DC
:100E300020E030E0C901E0960FB6F894DEBF0FBEA7
:100E4000CDBFCF91DF911F910F91FF90EF90DF9079
:100E5000CF90BF90AF909F908F907F906F905F905A
:100E60004F903F902F9008958091A2019091A301FF
:100E7000892BF1F64ECE1092A3011092A201D8CF89
:100E8000CF93DF939C01DB01009729F16115710578
:100E900011F11D968C911D9784FF1DC080914A0110
:100EA00090914B01892B19F4EAE4F1E008C080919C
:100EB000660190916701892B71F4E6E6F1E0EF019C
:100EC000229688E10D9009928150E1F731832083C9
:100ED000138E128E02C0E0E0F0E0CF01DF91CF91DF
:100EE00008952F923F924F925F926F927F928F92CE
:100EF0009F92AF92BF92CF92DF92EF92FF920F93A9
:100F00001F93DF93CF93CDB7DEB72A970FB6F89430
:100F1000DEBF0FBECDBF4C017C836B831A010097EF
:100F200009F4DEC0672B09F4DBC04115510509F453
:100F3000D7C0DC015A96ED90FD900D911C915D9704
:100F400080E09EEFAFEFBFEFE822F9220A231B23D8
:100F5000D4015A96ED92FD920D931C935D97529693
:100F60002D913D914D915C9155972E153F05400770
:100F7000510708F4B8C0C101A0E0B0E08E0D9F1D7C
:100F8000A01FB11F281739074A075B0728F419016A
:100F90002E183F0809F4A7C0D401ED91FC911197D8
:100FA000208931893A8329835E968D919C915F9740
:100FB0009A878987290166247724892BD9F5509649
:100FC0000D90BC91A02DBA87A987AB2B39F4E11401
:100FD000F1040105110509F486C082C0E114F10491
:100FE0000105110539F15701680188279927DC01AE
:100FF00084199509A609B7098D839E83AF83B887A5
:1010000014C069857A85D4018D919C910E94D70284
:101010009A878987892B09F463C08D819E81AF816E
:10102000B885A80EB91ECA1EDB1EA414B504C604DA
:10103000D70438F7510191E0291692E0390618F0EB
:10104000A12C82E0B82EC801B701A30192010E9431
:101050000B177B0129813A81261B370B65012A1565
:101060003B0508F4690100E010E0D401ED91FC912A
:1010700086899789A08DB18DE80EF91E0A1F1B1F66
:10108000E985FA853297BF0180E090E03296FA87D1
:10109000E987A30192010E94C516E60EF71E081FFC
:1010A000191F96014B815C81C801B7010E946E0C2B
:1010B000892BC9F0960140E050E0F401828D938DB8
:1010C000A48DB58D820F931FA41FB51F828F938FA0
:1010D000A48FB58F29853A85378F268FA50105C046
:1010E0004FEF5FEF02C040E050E0CA012A960FB612
:1010F000F894DEBF0FBECDBFCF91DF911F910F914E
:10110000FF90EF90DF90CF90BF90AF909F908F9027
:101110007F906F905F904F903F902F900895CF9366
:10112000DF939C01FB01009731F06115710519F007
:10113000858584FF2CC060E08CE790E003C060E010
:1011400088E690E00E94D70C20E030E0C901DF91F2
:10115000CF910895C4E8D1E0DF0188E10D900992B4
:101160008150E1F7309383012093820110929C011A
:1011700010929D0110929E0110929F018685978585
:101180009093A1018093A00122E831E0DFCF80910C
:10119000820190918301892B91F6DCCFFC010097AD
:1011A00011F480E00895108681E008958F929F9257
:1011B000AF92BF92CF92DF92EF92FF920F93DF93A5
:1011C000CF93CDB7DEB760970FB6F894DEBF0FBEF2
:1011D000CDBF7C016B015A014901009709F493C00E
:1011E0006115710509F48FC004300CF08CC007FD47
:1011F0001DC0602F772767FD7095E4E0660F771FAD
:10120000EA95E1F762547E4F882777FD8095982F05
:1012100020E130E0AE014F5F5F4FF7010995882371
:1012200009F471C08D81882309F46DC08091C401D7
:10123000882309F068C07CC08D818093C4012A8511
:1012400030E040E050E0542F432F322F22278B858F
:1012500090E0A0E0B0E0DC0199278827282B392B0B
:101260004A2B5B2B898590E0A0E0B0E0282B392B3E
:101270004A2B5B2B8C8590E0A0E0B0E0B82FAA272A
:1012800099278827282B392B4A2B5B2B2093C501C4
:101290003093C6014093C7015093C8012E8530E0BA
:1012A00040E050E0542F432F322F22278F8590E0CB
:1012B000A0E0B0E0DC0199278827282B392B4A2BA6
:1012C0005B2B8D8590E0A0E0B0E0282B392B4A2BDA
:1012D0005B2B888990E0A0E0B0E0B82FAA2799277F
:1012E0008827282B392B4A2B5B2B2093C90130935D
:1012F000CA014093CB015093CC0103C08FEF809380
:10130000C4019F0102C020E030E0C90160960FB621
:10131000F894DEBF0FBECDBFCF91DF910F91FF904C
:10132000EF90DF90CF90BF90AF909F908F900895F7
:10133000ECEBF1E081E1DF011D928A95E9F7F09293
:10134000BD01E092BC01D092BF01C092BE01B0923B
:10135000C101A092C0019092C3018092C20107FF17
:101360006BCFCCCF81E0089581E00895282F8FEFD7
:101370008EBD0DB407FEFDCF8DB58F778DBD8EB5BB
:10138000822F80648EBD0DB407FEFDCF8DB58F77A3
:101390008DBD872F9927AA27BB278EBD0DB407FEC9
:1013A000FDCF8DB58F778DBDCB01AA27BB278EBD15
:1013B0000DB407FEFDCF8DB58F778DBDBB27A72F51
:1013C000962F852F8EBD0DB407FEFDCF8DB58F777F
:1013D0008DBD4EBD0DB407FEFDCF8DB58F778DBD94
:1013E000222311F08FEF01C085E98EBD0DB407FEF9
:1013F000FDCF8DB58F778DBD90E02FEF2EBD0DB455
:1014000007FEFDCF8DB58F778DBD8EB58F3F19F45B
:101410009F5F9A3099F70895CF93DF93239A259A87
:10142000229A24982A9A83E58CBD8DB58E7F8DBD36
:1014300020E030E09FEF9EBD0DB407FEFDCF8DB5DF
:101440008F778DBD8EB52F5F3F4F2A30310599F7CD
:101450002A98C0E0D0E040E050E060E070E080E03A
:101460000E94B609813031F081E0CF3FD807E1F02A
:101470002196F1CFC0E0D0E040E050E060E070E0C5
:1014800081E00E94B60980FF06C08FE7CF3FD807F2
:1014900059F02196F1CF40E052E060E070E080E149
:1014A0000E94B609882319F02A9A80E008C02A9A77
:1014B0008CB58C7F8CBD8DB581608DBD81E0DF9159
:1014C000CF9108958F929F92AF92BF92DF92EF9249
:1014D000FF920F931F93CF93DF937B018C015A01EF
:1014E000E901DD24DA94812C42E0942E5EC02A9832
:1014F000B801A70140705E7F81E10E94B609882390
:1015000019F02A9A80E055C0DEBC0DB407FEFDCF6D
:101510008DB58F778DBD8EB58E3FB1F7A701517018
:10152000B401641B750BC617D70708F4BE01FB0195
:10153000E40FF51F20E030E0DEBC0DB407FEFDCF68
:101540008DB58F778DBD8EB52417350730F02E17EA
:101550003F0718F4D5018D935D012F5F3F4FB2E037
:1015600020303B0749F7DEBC0DB407FEFDCF8DB53B
:101570008F778DBD8EB5DEBC0DB407FEFDCF8DB56A
:101580008F778DBD8EB52A9ADEBC0DB407FEFDCFD8
:101590008DB58F778DBD8EB5C61BD70BCB01A0E067
:1015A000B0E0E80EF91E0A1F1B1F209709F09FCF1D
:1015B00081E0DF91CF911F910F91FF90EF90DF902D
:1015C000BF90AF909F908F9008952091000130912F
:1015D00001019FEF0AC09EBD0DB407FEFDCF8DB582
:1015E0008F778DBD8EB52F5F3F4F82E0203038075B
:1015F00090F38FEF8EBD0DB407FEFDCF8DB58F77C5
:101600008DBD8EB58FEF8EBD0DB407FEFDCF8DB5B0
:101610008F778DBD8EB52A9A8FEF8EBD0DB407FEE4
:10162000FDCF8DB58F778DBD8EB58FEF9FEF9093EA
:1016300001018093000108952F923F924F925F9293
:101640006F927F928F929F92AF92BF92CF92DF92D2
:10165000EF92FF920F931F93DF93CF93CDB7DEB737
:101660002C970FB6F894DEBF0FBECDBF4B015C01C7
:101670001A013C872B872801FE82ED82D886CF8213
:101680004115510509F4DAC02115310509F4D6C018
:101690000217130708F4D2C0EF2809F4CFC02A9824
:1016A000309521953F4F3A87298784011170D501E4
:1016B000C40180709E7F89839A83AB83BC83AC0115
:1016C000BD0181E10E94B609882311F02A9AB6C0B3
:1016D0009FEF9EBD0DB407FEFDCF8DB58F778DBDFD
:1016E0008EB58E3FA9F720E030E00BC0AFEFAEBD66
:1016F0000DB407FEFDCF8DB58F778DBD8EB52F5FF5
:101700003F4F2017310790F3E12C52E0F52EE01AFD
:10171000F10A3701EB85FC856E1A7F0A6201CE1A49
:10172000DF0A00E012E00E191F092B853C85E21646
:10173000F30648F14216530630F1F10120E030E0A3
:101740000CC08FEF8EBD0DB407FEFDCF8DB58F772A
:101750008DBD8EB581932F5F3F4FAB85BC852A171A
:101760003B0778F3A80160E070E0480D591D6A1D41
:101770007B1D2F813885C101ED81FE81099588236C
:1017800021F491E026C090E024C02B853C85E21A2C
:10179000F30A421A530A61147104A9F389859A85E0
:1017A000680E791EC80ED91E020F131FC9018C0DB9
:1017B0009D1D892B09F0B9CFE6CFAFEFAEBD0DB4BB
:1017C00007FEFDCF8DB58F778DBD8EB50894E108EE
:1017D000F108E114F10489F7BFEFBEBD0DB407FEB7
:1017E000FDCF8DB58F778DBD8EB5EFEFEEBD0DB40E
:1017F00007FEFDCF8DB58F778DBD8EB52B853C85D2
:101800004216530678F0992369F489809A80AB8058
:10181000BC8080E092E0A0E0B0E0880E991EAA1E95
:10182000BB1E43CF2A9A8FEF8EBD0DB407FEFDCFAE
:101830008DB58F778DBD8EB581E001C080E02C968F
:101840000FB6F894DEBF0FBECDBFCF91DF911F91D1
:101850000F91FF90EF90DF90CF90BF90AF909F904F
:101860008F907F906F905F904F903F902F90089552
:10187000FC0120910001309101014FEF2F3F34070F
:1018800031F460E086E890E00E94D70CFFCFCB01F6
:10189000820F931F8150924020F060E072E0621B43
:1018A000730B20E030E04FEF14C04EBD0DB407FEC7
:1018B000FDCF8DB58F778DBD8EB581938091000161
:1018C00090910101019690930101809300012F5F97
:1018D0003F4F2617370748F3CB010895CF92DF9289
:1018E000EF92FF920F931F93CF93DF937B018C01B5
:1018F0006A0180910001909101018F5F9F4F31F04B
:1019000060E08BE890E00E94D70CFFCFE90182E015
:101910002130380710F0C0E0D2E02A9880E09EEF36
:10192000AFEFBFEFE822F9220A231B23B801A7017A
:1019300081E10E94B609882321F02A9AC0E0D0E014
:101940002CC09FEF9EBD0DB407FEFDCF8DB58F77E8
:101950008DBD8EB58E3FB1F710920101109200013E
:101960002FEF14C02EBD0DB407FEFDCF8DB58F77C0
:101970008DBD8EB5D6018D936D0180910001909142
:101980000101019690930101809300018091000173
:10199000909101018C179D0728F3CE01DF91CF9123
:1019A0001F910F91FF90EF90DF90CF9008950F93CC
:1019B0001F93CF93DF93EC01062F10E005C08DEF4E
:1019C00093E00E94C7121F5FFE01E10FF11D6491B9
:1019D0006623A9F7002351F06AE08DEF93E00E949F
:1019E000CF126DE08DEF93E00E94CF12DF91CF9187
:1019F0001F910F9108951F920F920FB60F9211240D
:101A00002F933F934F938F939F93AF93BF93EF93F6
:101A1000FF93E091CD01F091CE01309709F4A8C079
:101A20002091D3033091D4038091D5039091D603B4
:101A30002817390709F047C08091D8038823B9F1E6
:101A40008091CF039091D0032FEC32E041E08F3CA6
:101A5000940749F43093D0032093CF039093D2039B
:101A60008093D1030AC08FEC91E09093D0038093D0
:101A7000CF033093D2032093D1038091CF03909171
:101A8000D0039093D4038093D30380509F4F9093BF
:101A9000D6038093D5031092D8038091D70388236F
:101AA00091F480916F00846080936F000CC08189F5
:101AB0009289A389B4890196A11DB11D818B928B56
:101AC000A38BB48B55C05A985C985B9A5B985C9AD0
:101AD0005B9A5B985B9A5B985B9A5B988781803195
:101AE00019F5E091D303F091D4038181805890E0FF
:101AF00087FF02C05C9A01C05C985B9A5B989F5F0D
:101B0000983011F0880FF4CF908180E097FF02C0E9
:101B10005C9A01C05C985B9A5B988F5F843011F08F
:101B2000990FF4CF32961DC08830F9F4E091D303B9
:101B3000F091D403908180E097FF02C05C9A01C0CD
:101B40005C985B9A5B988F5F883011F0990FF4CFA7
:101B50005B9A5B985B9A5B985B9A5B985B9A5B98E5
:101B60003196F093D403E093D3035A9A5D985D9A2B
:101B7000FF91EF91BF91AF919F918F914F913F91C5
:101B80002F910F900FBE0F901F90189508950895F4
:101B9000DC015696ED91FC9157976289738984898F
:101BA000958908959A01AB0160E074E284EF90E0BA
:101BB0000E940B1730938900209388000895CF93DB
:101BC000DF93EC0180916F008D7F80936F008D8992
:101BD000882319F00E94E50A1D8AE091CD01F09159
:101BE000CE01108A1092CE011092CD01DF91CF91DB
:101BF00008950F931F93DF93CF9300D000D0CDB7FC
:101C0000DEB78C01407049835A836B837C83DC018F
:101C100050968C91882351F0F894F8018589882397
:101C200029F00E94E50AD80155961C9240E0BE01B9
:101C30006F5F7F4FF801868997890E946404D801FD
:101C40005696ED91FC91579782899389A489B5891D
:101C500029813A814B815C81821B930BA40BB50BCC
:101C6000F80180879187A287B38778940F900F90AF
:101C70000F900F90CF91DF911F910F910895CF9208
:101C8000DF92EF92FF920F931F93DF93CF93CDB725
:101C9000DEB728970FB6F894DEBF0FBECDBF8C011C
:101CA0006B0144E050E07E010894E11CF11CB70197
:101CB000C6010E942103049709F0F0C044E050E0FF
:101CC00062E071E0C7010E94A816009709F0E6C023
:101CD000F5C044E050E067E071E0CE0105960E9457
:101CE000A816009709F0DAC0F2C044E050E06CE0BA
:101CF00071E0C7010E94A816009709F0CFC0F0C09C
:101D0000542F432F322F22278081280F311D411D50
:101D1000511D3197EC17FD0799F7F8012487358796
:101D200046875787203131054105510509F0B6C076
:101D300048E050E0BE016F5F7F4FC6010E94210363
:101D4000089709F0ABC08A8190E0A0E0B0E0BA2F1C
:101D5000A92F982F88272981820F911DA11DB11DC0
:101D60000197A105B10521F061E088EA90E084C007
:101D70008C8190E0A0E0B0E02227382F492F5A2F25
:101D80008B81280F311D411D511D23303105410527
:101D9000510508F083C0F8012083FE013896BE018A
:101DA0006C5F7F4F542F432F322F22278081280FC3
:101DB000311D411D511D3197E617F70799F7F801BD
:101DC000218332834383548348E050E0BE016F5F38
:101DD0007F4FC6010E942103089709F05FC08E81E2
:101DE00090E0A0E0B0E0BA2FA92F982F88272D818E
:101DF000820F911DA11DB11DF801968385838885F1
:101E000090E0A0E0B0E02227382F492F5A2F8F8191
:101E1000280F311D411D511D21313105410551054D
:101E200008F03CC0278381819281A381B4818332F1
:101E3000F6E59F07F0E0AF07F0E0BF0718F02930A4
:101E400040F00CC081589E43A040B04050F0293073
:101E500040F0FF24F8018081823020F0FF24F394C9
:101E600001C0FF2461E087EA90E00E94D70CFF20C8
:101E700031F061E081E990E00E94D70C0FC0F801D9
:101E80001086118612861386D78AC68A118A128A0C
:101E9000138A148A108A158A81E001C080E028968E
:101EA0000FB6F894DEBF0FBECDBFCF91DF911F916B
:101EB0000F91FF90EF90DF90CF90089548E050E0B1
:101EC000B701C6010E942103089741F702CF44E001
:101ED00050E0B701C6010E9421030497F9F605CF2F
:101EE000F801148615861686178644E050E0B7017F
:101EF000C6010E942103049789F6F80124853585DF
:101F000046855785FE013496FBCEAF92BF92CF92A5
:101F1000DF92EF92FF920F931F93DF93CF9300D046
:101F200000D00F92CDB7DEB76C015B01F42EE52E29
:101F3000FC0180859185A285B3850097A105B10537
:101F4000D1F544E050E08E010F5F1F4FB801868944
:101F500097890E942103049709F0F5C01D8244E08F
:101F600050E0B801D60156968D919C9157970E94EA
:101F70002103049709F0E7C0F60110861186128646
:101F80001386FE01349620E030E040E050E0542F0C
:101F9000432F322F22278081280F311D411D511DD3
:101FA0003197EC17FD0799F7D60118962D933D93BD
:101FB0004D935C931B978F2D9E2D9C017901B2E070
:101FC00021303B0718F0E12C72E0F72EF601208556
:101FD000318542855385C701A0E0B0E02817390755
:101FE0004A075B0708F47901D6015696ED91FC91FA
:101FF0005797828D938DA48DB58D9170A070B07020
:102000000097A105B105D1F4D60155968C9188238E
:10201000A9F4A701B501CF010E9471078C018E15AB
:102020009F0541F060E082EE90E00E94D70C0E9494
:10203000E50A8BC081E0F601858B73C0D601559609
:102040008C91882309F463C0B701C5010E94380C44
:102050005C018E159F0539F060E08CED90E00E94E8
:10206000D70C0E94E50AD6015696ED91FC91579740
:10207000C501A0E0B0E0228D338D448D558D820FD7
:10208000931FA41FB51F828F938FA48FB58F91705C
:10209000A070B0700097A105B10509F041C00E9481
:1020A000E50AF601158A06891789D801ED90FC909A
:1020B0001197F7012089318940E050E05A966D91DF
:1020C0007D918D919C915D970E940B176115710513
:1020D0008105910529F5D8015E966D917C915F97F8
:1020E000C7010E94D702F801978F868F892BC1F410
:1020F000D6015696ED91FC915797178E168E61E09A
:1021000082EC90E00E94D70C0FEF1FEF1EC0A701DA
:10211000B501CF010E9421038E159F05A1F401C0D6
:102120007501970140E050E0F60180859185A28518
:10213000B385821B930BA40BB50B80879187A28775
:10214000B387870102C000E010E0C8010F900F9034
:102150000F900F900F90CF91DF911F910F91FF90F3
:10216000EF90DF90CF90BF90AF900895CF92DF9225
:10217000EF92FF920F931F93CF93DF93EC01C980EF
:10218000DA80EB80FC809093CE018093CD010FEC40
:1021900011E01093D4030093D30342E050E0B80160
:1021A0000E94850F892B09F451C08091D30390912F
:1021B000D40302969093D6038093D503EE89FF89CA
:1021C000828D40E051E0481B5109B8016E5F7F4F9E
:1021D0008091CD019091CE010E94850F9C010097C6
:1021E000A9F18091D5039091D603820F931F90930C
:1021F000D6038093D50340E051E06FEC72E080910C
:10220000CD019091CE010E94850F81E08093D8038B
:10221000888B1092800089E08093810060E074E2F6
:1022200084EF90E0A70196010E940B17309389007C
:102230002093880081E090E090938B0080938A0047
:1022400080916F00826080936F007894DF91CF91CE
:102250001F910F91FF90EF90DF90CF9008951F9204
:102260000F920FB60F9211242F933F934F935F93CA
:102270006F937F938F939F93AF93BF93EF93FF934E
:1022800080916F008B7F80936F008091D8038823AB
:10229000F9F481E08093D70378946091D103709131
:1022A000D20340E051E08091CD019091CE010E9497
:1022B000850F892B31F48091CD019091CE010E9440
:1022C000DF0DF8941092D70381E08093D8037894BF
:1022D000FF91EF91BF91AF919F918F917F916F91FE
:1022E0005F914F913F912F910F900FBE0F901F90D4
:1022F00018958BED93E00E94F80083EE93E00E9426
:10230000C70D08950F931F9383EE93E00E94DF0D96
:102310006091E1037091E2030BED13E0C8010E94AC
:10232000F900C8010E94FD001F910F910895CF93FD
:10233000DF93EC018091F303882361F083EE93E057
:102340000E94DF0D6091E1037091E2038BED93E059
:102350000E94F9008BED93E00E94FD00BE018BED21
:1023600093E00E945301BC019093E2038093E10348
:10237000009751F083EE93E00E943F0E882321F0F6
:1023800083EE93E00E94B610DF91CF9108950E94F2
:1023900097118091F3038823E1F76091E103709135
:1023A000E2038BED93E00E94F90008951F938DEFF7
:1023B00093E00E94BF12882389F08DEF93E00E9482
:1023C000BC12182F482F50E060E070E020E030E0B1
:1023D0008DEF93E00E943614812F00C01F91089565
:1023E0000E94D6118093FC038330C9F084303CF402
:1023F000813079F0823084F4882341F0089585306B
:10240000A1F085307CF08630C9F414C00E9482119E
:10241000089581E191E00BC087E191E008C08DE172
:1024200091E005C083E291E002C089E291E00E9460
:10243000C71108958FE291E00E94C71108950F938C
:102440001F93DF93CF93CDB7DEB72D970FB6F894D8
:10245000DEBF0FBECDBF8BED93E00E94FD0061E0BB
:1024600088EE90E00E94D70C8E010F5F1F4FB801DD
:102470008BED93E00E945C01882379F48BED93E06F
:102480000E94FD002D960FB6F894DEBF0FBECDBFA3
:10249000CF91DF911F910F910895B8018DEF93E0D7
:1024A0000E941613E4CF40E855E260E070E08DEF43
:1024B00093E00E94C21265E371E08DEF93E00E9409
:1024C000161361E082E00E94331561E083E00E9410
:1024D000331561E084E00E94331561E085E00E94DD
:1024E000331561E089E00E9433158BED93E00E9483
:1024F0000502882321F461E088E391E01DC08BEDA3
:1025000093E00E94DA01882321F461E08AE291E0FD
:1025100013C08BED93E00E94C701882321F461E092
:1025200084E191E009C08BED93E00E949301882340
:1025300031F461E082E091E00E94D70C089561E0FF
:1025400085EF90E00E94D70C0E941F1208950E9410
:10255000F9140E9453120E94F011FDCF88E491E01B
:102560009093FE038093FD030895862F0E94211609
:1025700008950E94591608950E943A1608950E94DF
:1025800029160895CB01BA010E94E8150895DC01CF
:10259000ED91FC910190F081E02D09950895DC0109
:1025A000ED91FC910190F081E02D099508950F9334
:1025B0001F93CF93DF938C01EB0109C02196D801C3
:1025C000ED91FC910190F081E02DC80109956881A1
:1025D0006623A1F7DF91CF911F910F9108950F937B
:1025E0001F938C01DC01ED91FC910190F081E02DB5
:1025F0006DE00995D801ED91FC910190F081E02DFD
:102600006AE0C80109951F910F9108950F931F93D8
:102610008C01DC01ED91FC910190F081E02D099598
:10262000C8010E94EF121F910F9108950F931F93FD
:102630008C010E94D712C8010E94EF121F910F91C6
:1026400008950F931F938C01DC01ED91FC91019093
:10265000F081E02D0995C8010E94EF121F910F91A2
:1026600008952F923F924F925F926F927F928F9236
:102670009F92AF92BF92CF92DF92EF92FF920F9311
:102680001F93DF93CF93CDB7DEB7A0970FB6F89423
:10269000DEBF0FBECDBF1C016A017B014115510594
:1026A0006105710549F4DC01ED91FC910190F08127
:1026B000E02D60E3099554C0882499245401422EEA
:1026C00055246624772401E010E00C0F1D1F080D2F
:1026D000191DC701B601A30192010E940B17F80151
:1026E00060830894811C911CA11CB11CC701B60118
:1026F000A30192010E940B17C901DA016C017D014F
:10270000C114D104E104F104F1F681E0E82EF12CCA
:10271000EC0EFD1EE80CF91C3E010894611C711CB6
:10272000D501C4010197A109B1096C01C818D908E4
:1027300014C0F601EE0DFF1D60816A3010F4605D7B
:1027400001C0695CD101ED91FC910190F081E02D17
:10275000C10109950894E108F1086E147F0449F756
:10276000A0960FB6F894DEBF0FBECDBFCF91DF911C
:102770001F910F91FF90EF90DF90CF90BF90AF909F
:102780009F908F907F906F905F904F903F902F9091
:1027900008952AE00E94311308950F931F938C012E
:1027A0000E94C913C8010E94EF121F910F91089552
:1027B000AB0160E070E00E94C91308950F931F936E
:1027C0008C01AB0160E070E00E94C913C8010E9457
:1027D000EF121F910F910895EF92FF920F931F93A5
:1027E000CF93DF93EC017A018B0177FF0FC0E88173
:1027F000F9810190F081E02D6DE209951095009529
:10280000F094E094E11CF11C011D111D2AE0B801B7
:10281000A701CE010E943113DF91CF911F910F913B
:10282000FF90EF9008950F931F938C010E94EC137B
:10283000C8010E94EF121F910F910895AB01662706
:1028400057FD6095762F0E94EC1308950F931F9308
:102850008C01AB01662757FD6095762F0E94EC1323
:10286000C8010E94EF121F910F910895DC012115FC
:10287000310541F4ED91FC910190F081E02D642F40
:10288000099508952A30310519F40E94EC13089532
:102890000E94311308950F931F938C010E943614E8
:1028A000C8010E94EF121F910F9108951F920F927D
:1028B0000FB60F9211242F938F939F93AF93BF93D3
:1028C0008091FF0390910004A0910104B091020453
:1028D0008050904CAF4FBF4F8093FF039093000404
:1028E000A0930104B093020427C08091FF0390914C
:1028F0000004A0910104B091020480589E43A040BE
:10290000B0408093FF0390930004A0930104B09320
:1029100002048091030490910404A0910504B091F5
:1029200006040196A11DB11D809303049093040435
:10293000A0930504B09306048091FF0390910004D6
:10294000A0910104B091020481589E43A040B04080
:1029500060F6BF91AF919F918F912F910F900FBE15
:102960000F901F9018958FB7F89420910304309121
:10297000040440910504509106048FBFB901CA01B7
:102980000895EF92FF920F931F937B018C018FB7F5
:10299000F8944091030450910404609105047091EF
:1029A00006048FBF2FB7F89480910304909104041C
:1029B000A0910504B09106042FBF841B950BA60BB4
:1029C000B70B8E159F05A007B10760F31F910F91FC
:1029D000FF90EF900895019759F0FC01EE0FFF1F53
:1029E000EE0FFF1F32978FB7F8943197F1F78FBF33
:1029F0000895789484B5826084BD84B5816084BD77
:102A000085B5826085BD85B5816085BDEEE6F0E067
:102A1000808181608083E1E8F0E080818260808352
:102A2000808181608083E0E8F0E080818160808344
:102A3000E1EBF0E0808184608083E0EBF0E0808176
:102A400081608083EAE7F0E0808184608083808118
:102A500082608083808181608083808180688083C0
:102A60001092C1000895282F30E0C90182599E4F6D
:102A7000FC019491265A3E4FF9018491882381F0FC
:102A8000E82FF0E0E55BFE4FE491F0E0662329F4E7
:102A9000808190958923808308958081892B80830C
:102AA0000895482F50E0CA018E579E4FFC01249193
:102AB000CA0182599E4FFC019491465A5E4FFA0119
:102AC00034913323C1F1222331F1233021F4809159
:102AD00080008F7705C0243031F4809180008F7D95
:102AE0008093800018C0213019F484B58F7704C01A
:102AF000223021F484B58F7D84BD0DC0263021F4B1
:102B00008091B0008F7705C0273029F48091B00004
:102B10008F7D8093B000E32FF0E0E05BFE4FE49107
:102B2000F0E0662329F480819095892380830895BD
:102B30008081892B80830895482F50E0CA018E57E9
:102B40009E4FFC012491CA0182599E4FFC01949131
:102B5000465A5E4FFA013491332319F420E030E0F5
:102B600035C0222331F1233021F4809180008F770A
:102B700005C0243031F4809180008F7D80938000E7
:102B800018C0213019F484B58F7704C0223021F4A5
:102B900084B58F7D84BD0DC0263021F48091B000B6
:102BA0008F7705C0273029F48091B0008F7D809306
:102BB000B000E32FF0E0EB5AFE4FE491F0E08081AB
:102BC00020E030E0892311F021E030E0C9010895D0
:102BD000EF92FF920F931F937B018C0122E030E074
:102BE00040E050E00E942D17205C3D4B404F5F4F6E
:102BF000CA01B901A80197010E942D17C901DA0184
:102C00000197A109B109292F3A2F4B2F552747FDCD
:102C10005A950196A11DB11D2093C5008150809346
:102C2000C400E1ECF0E08081806180838081886075
:102C300080838081806880831F910F91FF90EF9047
:102C40000895982F8091C00085FFFCCF9093C60017
:102C50000895809107049091080480589F4F209117
:102C6000090430910A04821B930B60E870E00E9413
:102C7000F81608954091090450910A0480910704C0
:102C8000909108048417950719F42FEF3FEF0FC0B8
:102C9000FA01E55FFB4F2081CA01019660E870E010
:102CA0000E94F81690930A048093090430E0C90149
:102CB00008958091090490910A04909308048093E8
:102CC000070408951F920F920FB60F9211242F93AD
:102CD0003F934F935F936F937F938F939F93AF93A4
:102CE000BF93EF93FF934091C600E0910704F091EA
:102CF0000804CF01019660E870E00E94F8169C017C
:102D00008091090490910A042817390739F0E55F8A
:102D1000FB4F40833093080420930704FF91EF9109
:102D2000BF91AF919F918F917F916F915F914F91E3
:102D30003F912F910F900FBE0F901F901895FB01A0
:102D4000DC018D91019080190110D9F3990B089540
:102D5000FB01DC014150504030F08D910190801911
:102D600019F40020B9F7881B990B0895FB01DC01C9
:102D70004150504048F001900D920020C9F701C029
:102D80001D9241505040E0F70895629FD001739F1B
:102D9000F001829FE00DF11D649FE00DF11D929FF7
:102DA000F00D839FF00D749FF00D659FF00D992736
:102DB000729FB00DE11DF91F639FB00DE11DF91F5A
:102DC000BD01CF0111240895AA1BBB1B51E107C00F
:102DD000AA1FBB1FA617B70710F0A61BB70B881FAB
:102DE000991F5A95A9F780959095BC01CD0108953A
:102DF00097FB092E07260AD077FD04D0E5DF06D021
:102E000000201AF4709561957F4F0895F6F790951C
:102E100081959F4F0895A1E21A2EAA1BBB1BFD01AD
:102E20000DC0AA1FBB1FEE1FFF1FA217B307E407A9
:102E3000F50720F0A21BB30BE40BF50B661F771F01
:102E4000881F991F1A9469F76095709580959095E1
:102E50009B01AC01BD01CF01089597FB092E05260A
:102E60000ED057FD04D0D7DF0AD0001C38F450959F
:102E70004095309521953F4F4F4F5F4F0895F6F79E
:102E800090958095709561957F4F8F4F9F4F0895D6
:102E9000EE0FFF1F0590F491E02D0994F894FFCFF9
:102EA000FFFF52494646005741564500666D742063
:102EB00000312E57415600322E57415600332E57BF
:102EC000415600342E57415600352E574156003694
:102ED0002E5741560041756469666F6E6F207465A8
:0A2EE0007374210000000000B51219
:00000001FF
